:100E210025302E3166000313010A210004FFFFFF64
:100E3100FFFFFF0A210006FFFFFFFFFFFF0E230058
:100E410005FFFFFFFFFFFF523020100A240005FFBE
:100E5100FFFFFFFFFF0E250005FFFFFFFFFFFF0262
:100E61000000000E260005FFFFFFFFFFFF0200004C
:0B0E71000002126D6F6E6579203D00DD
:100E7C00024F02030927093100000411001100057B
:100E8C002205300000041A9A1A220004FFFFFFFF0B
:100E9C00FFFF06000000000000000000000102033C
:020EAC0004053B
:0F0EAF00C2A3C2A48F807F017E00120EBED2A408
:100EBE00E4FDFCC3ED9FEC9E5015E4FBFA0BBB006A
:0F0ECE00010AEB64644A70F50DBD00010C80E46D
:010EDD0022F2
:08104200C2A2120EAFC2A422EB
:08104A00D2A2120EAFC2A422D3
:100F38008B668A678968AB66AA67A9681205F0FF9D
:100F4800601712104A74012568F568E43567F5677B
:0A0F58007F017E00120EBE80DD2234
:100FF6007F381210427F801210427F061210427F05
:091006000C1210427F010210429D
:10102500120F387F88121042AB63AA64A965020FBC
:011035003882
:100F89007FFF120FD3AB60AA61A962856382758363
:090F990000EF1206487F0A7E00F9
:0C0FA200EF4E6007EF1F70F81E80F52274
:080EDE007812A6077F647E0074
:100EE60075CBFC75CA6975CDFC75CC69C2AD75C884
:100EF60004EF1FAC0670011E4C600730CFFDC2CF59
:050F060080EFC2CA22C9
:100F0B0075CBDC75CA0075CDDC75CC00C2AD75C870
:100F1B0004EF1FAC0670011E4C600F20CF08300A87
:0D0F2B00FAC2CAC2CF22C2CF80E7C2CA22DA
:100FD3007D08AC051DEC6016EE2EFEC295EF339234
:100FE30097EF2FFFA296E4334206D29580E4D29581
:020FF300AF0647
:010FF50022D9
:10100F00C2937FAA120FD37F327E00120FA27FFFEF
:05101F00120FD3D29373
:0110240022A9
:0D0C92007F647E00120EE67B007A00797C04
:060C9F008B608A6189628E
:100CA500E4F564F56312100FBFF0037563FD7F3241
:100CB5007E00120FA20563E563C3946440E7E56314
:100CC50064FE706CC2937FBB120FD38F63AB60AAB7
:100CD50061A9627401120636E4F563AB60AA61A9E5
:100CE500621205F0FFE563C39F5025120F89AB60C3
:100CF500AA61A9628563827583001206096264127E
:100D050005F0D394204005D2937F0122056380CB63
:100D1500120F9E120F89D293AB60AA61A9628563F7
:100D250082758300120609B564037F00227F0122C4
:020D35007F013C
:010D37002299
:100DC40078A47C007D007B007A00795C7E007F043F
:0F0DD4001205CA7B007A00799A8B598A5A895B7B
:060DE3008B608A61896249
:100DE900E4F564C2937FCC120FD3E4F563AB60AA38
:100DF90061A9621205F0FEE563C39E501385638203
:100E0900758300120609FF6264120FD3056380DD42
:070E1900AF64120FD3D29366
:010E200022AF
:0C103600C2927F327E00120F0BD2922279
:100B0F0078517C007D007BFF7A0E79747E007F0820
:100B1F001205CAE47813F608F6F55FF55E755DDD2C
:100B2F00755C42120FAE1210367FF47E01120EE684
:100B3F00120FF62094FD120DC47FF47E01120C9655
:100B4F007812A607AB59AA5AA95B900001120609A1
:100B5F00FF787DE6B507057812E6600B120DD71208
:100B6F000C92120EDE80DD7814E6640118467003D5
:100B7F00020C912094FD7F467E00120EE62094E732
:100B8F007BFF7A0E792A120DDD120C927812A607CE
:100B9F00AB59AA5AA95B900001120609FF787DE6AE
:100BAF00B507057812E6600F7BFF7A0E7972120D8A
:100BBF00E37812A60780C6785C7C007D007B007A04
:100BCF0000797E7E007F041205CAAF5FAE5EAD5D19
:100BDF00AC5CE4FBFA79C078BF12000A8F5F8E5EBF
:100BEF008D5D8C5CE4FFFEFDFCAB5FAA5EA95DA88A
:100BFF005C1200FB50167BFF7A0E7972120DE378B0
:100C0F0012A607087600087601020B76120DC412A1
:100C1F000C927812A607AB59AA5AA95B9000011241
:100C2F000609FF787DE6B507057812E6600B120D11
:100C3F00D7120C92120EDE80DD7563FF75640E7590
:100C4F006521855F69855E68855D67855C667B006C
:100C5F007A0079081206FC7BFF7A0E7972120DE387
:100C6F00120EE27563007564007565087B007A00EB
:100C7F0079511210257FD07E07120EE6120FF60261
:020C8F000B8CCC
:010C91002240
:100FAE00C2AD75C804758780759870758921758D69
:100FBE00FD858D8BD28EC2ABD2AFC2A8D288C2CAEB
:050FCE00D2ACC20A22B2
:1000030002019DE86480F8E933E83360110460F08D
:10001300ED33EC337009E8FCE9FDEAFEEBFF220463
:1000230060DED3EB9FEA9EE99DE8C2E78CF0C2F75E
:1000330095F0400CE8CCF8E9CDF9EACEFAEBCFFB2A
:1000430012016885D0F05804700320D5B3E804701A
:10005300075002B2D50201A792D5EC0460F7E4CCB5
:10006300C0E0C398F8603B94186008400DD0E0FBF3
:1000730002017FE4FBFAC9FC8028E830E406E4C906
:10008300FBE4CAFCE830E305E4C9CACBFCE8540747
:100093006010F8C3E913F9EA13FAEB13FBEC13FC52
:1000A300D8F130F52FC3E49CFCEF9BFFEE9AFEEDF5
:1000B30099FDD0E0FBEF4E4D4C701222DB030201A1
:1000C300A4EC2CFCEF33FFEE33FEED33FDED30E714
:1000D300EB02017FEF2BFFEE3AFEED39FDD0E0FBA3
:1000E30050130BBB00030201A7ED13FDEE13FEEF4C
:0800F30013FFEC13FC02017F76
:1000FB0074F8CC6480CCC86480C8F582046043C3B8
:10010B00EB9FF5F0EA9E42F0E99D42F0E89C45F04A
:10011B0060305018E5825FFFE582F42B5582FB506F
:10012B00210ABA001D09B90019088016E5825BFB8C
:10013B00E582F42F5582FF50090EBE00050DBD0060
:10014B00010CC3EB9FF5F0EA9E42F0E99D42F0E80B
:0D015B009C45F06007CC4820E701B3EC2282
:1006A000E5772463F8E605772278603007027863FF
:1006B000E475F00112066A0205F02000EB7F2ED2ED
:1006C000008018EF540F2490D43440D4FF30040B32
:1006D000EF24BFB41A0050032461FFE578600215CF
:1006E00078057BE57B7002057A30070D7860E4754C
:1006F000F00112066AEF020636020F627403D20797
:100700008003E4C207F5778B608A618962E4F5783B
:10071000F57AF57BE57860077F201206DB80F575BA
:1007200079FFC201C200C202C203C205C206C208EA
:100730001206A9FF700D3007057F001206ECAF7B93
:10074000AE7A22B4255FC2D5C2041206A9FF24D016
:10075000B40A00501A75F00A787830D50508B6FF4B
:100760000106C6A426F620D5047002D20380D9243F
:10077000CFB41A00EF5004C2E5D2040209D9D20165
:1007800080C6D20080C0D20280BCD2D580BAD20549
:1007900080B47F201206DB2002077401B578004088
:1007A000F11206A0FF1206DB020714D208D206805F
:1007B000951206A0FB1206A0FA1206A0F94A4B7089
:1007C0000679D07A0A7BFF20022EE578602A7E0027
:1007D0008E8275830012060960060EEE657970F050
:1007E000C2D5EBC0E0EAC0E0E9C0E0EE120A39D0C1
:1007F000E0F9D0E0FAD0E0FB1205F0FF60AAEBC010
:10080000E0EAC0E0E9C0E01206DBD0E02401F9D064
:10081000E03400FAD0E0FBE5790460DCD579D980DA
:1008200087D20280A2120A1C60F7E57970010412D7
:1008300001B2A979600DE579600914F579120AC34E
:10084000EF60F3EA30E702F404C3995077EAF42545
:10085000790430E701E404F579800D120A1C60C1C7
:10086000EA057925791201B2EA7876F630E701E4F3
:10087000257904D5790420050114120A39E4C0E071
:10088000120AC37876E6601320E70714F61206C34F
:10089000802204F6D0E014C0E07F001206C3E579A0
:1008A00060071206BA1579800B3005031206BAD01C
:1008B000E0020714D0E00480C5120A1C60A0E579AC
:1008C000041201B27876EAF6E579200502600104A7
:0508D0002404120A39A6
:1008D50074FF04C0E0120AC31206C3E579200502BD
:1008E50060031206BAD0E0B579E87F451206CD78E7
:1008F50076E67F2B30E7047F2DF404C0E01206DB9B
:10090500D0E075F00A84C0F01206C4D0E01206C427
:10091500020714791080027908C206C2088008D23D
:10092500D5790A8004790AC2D5E579047002F5798A
:10093500E4FAFDFEFF1206A0FC7B08200113120657
:10094500A0FD7B1030000A1206A0FE1206A0FF7B58
:1009550020EC3382D592D55013C3E43000069FFFB7
:10096500E49EFEE42001039DFDE49CFCE4CBF8C27B
:1009750001EC700CCFCECDCCE824F8F870F38017DD
:10098500C3EF33FFEE33FEED33FDEC33FCEB33FB0E
:10099500994002FB0FD8E9EB300105F8D0E0C448D7
:1009A500B201C0E00AEC4D4E4F78207B0070C2EAE0
:1009B500B5790040BCC0E0120A3BD0F0D0E0200180
:1009C50004C4C0E0C4B201C0F01206C4D0F0D5F032
:1009D500EB02071412067A07B15309185807824C1F
:1009E500077E42091C4F09244409244907974309F6
:1009F5002A55085B4608B9450825470AF050078679
:100A05002D078A2E07AD2B078E2307AB200AD92A7F
:100A1500074648000007A5E579B4FF037579061276
:100A250006A0FC1206A0FD1206A0FE1206A0FF7885
:100A35006F0201E1790AA2D5200314300509B91026
:100A4500020404B9080104A2D520060250010420BD
:100A550002689202B578005034C0E07F2030031957
:100A65007F30A20272067205500F120A92C202C2AC
:100A750006C205C2087F30800F300503E9C0E012C9
:100A850006DB300503D0E0F9D0E0B578CC300517AA
:100A95007F30B9100C1206DB7F583004077F788051
:100AA50003B908031206DB3002057F2D0206DB7F42
:100AB500202008F87F2B2006F322920280CF7F00AA
:100AC500B407005005246FF8E6FF22286E756C6C9C
:100AD5002900D2011206A03001F8C201787830D57C
:100AE5000108F60207462D504349581206A0240373
:100AF500B405004001E4900AEB931206CC743A1257
:0A0B050006CCD2037578040209182B
:10016800E9D2E7C933E833F892D5EDD2E7CD33ECDD
:0701780033FC5002B2D52256
:10017F00EC30E7100FBF000C0EBE00080DBD0004E1
:10018F000BEB6014A2D5EB13FCED92E7FD2274FF8D
:10019F00FCFDFEFF22E480F8A2D574FF13FC7D80E6
:0301AF00E480EFFA
:1001B200F920E72824F950037907E4F42402FB1814
:1001C200DBFDE624FB5014E9600DE4F618E604F6C4
:0F01D200B40A08E4F6D9F57401F60A22C2D52260
:1001E100ED33EC3392D5FA602AB4FF33EDC2E77BED
:1001F100FF60067A027906E4227A02790F20D5049B
:100201007A02790A224E614E002B494E46002D4951
:100211004E4600E47A08F608DAFC7B00740722E80F
:10022100C0E0ECC0E0EDC0E0EEC0E0EFC0E0EA7598
:10023100F010A4CAABF075F04DA42BFBE435F0FC33
:10024100EA2410FAEB34C5FBEC34D9FCEDC2E7FF2C
:1002510075F056A4F42411C5F0F434C58FF0A42A26
:10026100E5F03BE43CF620E7141204BAD0E0FFD0FD
:10027100E0FED0E0FDD0E0FC1203ED8014F40412A6
:1002810004BAD0E0FFD0E0FED0E0FDD0E0FC1202E5
:10029100E4D0E0F8E6FAEDD2E7CD33EC332482FB8B
:1002A100E4C3CF33CFCE33CECD33CD33DBF37B07B6
:1002B10075F00A846004F6081B0AE5F0F6088FF071
:1002C100740AA4FFACF08EF0740AA42CFEACF050BA
:1002D100010C8DF0740AA42CFDE435F0F608DBDE88
:0302E1007407227D
:1002E400EC4D6011E8497017ED33EC3304600DE414
:1002F400FCFFFEFD22E933E8330470F802019D128D
:10030400016858046009E4CC24815006285009028D
:1003140001A72840030201A4C0E0EB4A7044B9805D
:1003240006D0E0FB020193EF4E701CBD8008EBFF8A
:10033400EAFEE9FD80EBE98DF0A4FEE5F00203CDD1
:10034400E9CDF9EAFEEBFFEF89F0A4FCE5F0CE89F4
:10035400F0A42EFFE435F0CD89F0A42DFEE435F0B1
:100364008067EF4E7005BD80D780C3EF8BF0A4ACDF
:10037400F0EE8BF0A42CFCE435F0F8EF8AF0A42C1A
:10038400E5F038FCE433CB8DF0A42CFCE5F03BF82D
:10039400EE8AF0A42CFCE5F038F8E433CF89F0A41D
:1003A4002CFCE5F038CF3400CE89F0A42FFFE5F023
:1003B4003EFEE433C98DF0A42EFEE5F039CD8AF07B
:1003C400A42FFFE5F03EFEE43DFD33D0E0FB5007F3
:1003D4000BBB000F0201A7EC2CFCEF33FFEE33FE46
:0603E400ED33FD02017F74
:1003EA000201A7EC5D046005E85904700302019D4F
:1003FA00120168580460F6EC4860F2EC7004FDFEE5
:10040A00FF22C860DB2481C85009C39860025006E5
:10041A000201A49850CAF582E9294B4A7005AB82B9
:10042A0002019375F0007C1A7880C3EF9BEE9AED77
:10043A0099400DC3EF9BFFEE9AFEED99FDE842F05D
:10044A00DC23ACF0D0E0FFD0E0FED0E0FDAB8220B0
:10045A00E7101BEB60BAEC2CFCEF33FFEE33FEED3A
:10046A0033FD02017FE803F830E705C0F075F000BC
:10047A00EF2FFFEE33FEED33FD40B830E7C280AA1E
:10048A003F8000004120000042C80000447A00007A
:10049A00461C400047C35000497424004B189680FC
:1004AA004CBEBC205A0E1BCA6753C21C749DC5AEF3
:1004BA00FB60065407601C23231204E8EB543860DF
:1004CA00091204D41204E31202E4ECF8EDF9EEFA8C
:1004DA00EFCB22EB1204E380F1543803241C90047E
:1004EA008AFE93FC0EEE93FD0EEE930ECE93FF2240
:03000000020D38B6
:0C0D3800787FE4F6D8FD7581B7020D7FCE
:1004FA00E709F608DFFA8046E709F208DFFA803EE4
:10050A0088828C83E709F0A3DFFA8032E309F608D0
:10051A00DFFA8078E309F208DFFA807088828C8338
:10052A00E309F0A3DFFA806489828A83E0A3F608EC
:10053A00DFFA805889828A83E0A3F208DFFA804CC6
:10054A0080D280FA80C680D4806980F2803380109D
:10055A0080A680EA809A80A880DA80E280CA803306
:10056A0089828A83ECFAE493A3C8C582C8CCC5837E
:10057A00CCF0A3C8C582C8CCC583CCDFE9DEE7804E
:10058A000D89828A83E493A3F608DFF9ECFAA9F0CD
:10059A00EDFB2289828A83ECFAE0A3C8C582C8CC23
:1005AA00C583CCF0A3C8C582C8CCC583CCDFEADE3C
:1005BA00E880DB89828A83E493A3F208DFF980CC9E
:1005CA0088F0EF60010E4E60C388F0ED2402B40497
:1005DA000050B9F582EB2402B4040050AF2323453E
:0605EA00822390054A7314
:1005F000BB010689828A83E0225002E722BBFE0209
:09060000E32289828A83E493223B
:10060900BB010CE58229F582E5833AF583E02250A6
:1006190006E92582F8E622BBFE06E92582F8E222F0
:0D062900E58229F582E5833AF583E493220A
:10063600BB010689828A83F0225002F722BBFE01A3
:02064600F3229D
:10064800F8BB010DE58229F582E5833AF583E8F0E8
:10065800225006E92582C8F622BBFE05E92582C894
:02066800F2227C
:10066A00FAE6FB0808E6F925F0F618E6CA3AF62291
:10067A00D083D082F8E4937012740193700DA3A30F
:10068A0093F8740193F5828883E473740293686023
:06069A00EFA3A3A380DF23
:100F6200EFB40A07740D120F6D740A309811A89924
:100F7200B8130CC2983098FDA899C298B811F630EF
:070F820099FDC299F59922C7
:100D4400020B0FE493A3F8E493A34003F68001F2AB
:100D540008DFF48029E493A3F85407240CC8C333B0
:100D6400C4540F4420C8834004F456800146F6DF7F
:100D7400E4800B0102040810204080900E7CE47E85
:100D8400019360BCA3FF543F30E509541FFEE49374
:100D9400A360010ECF54C025E060A840B8E493A33B
:100DA400FAE493A3F8E493A3C8C582C8CAC583CA66
:100DB400F0A3C8C582C8CAC583CADFE9DEE780BE1E
:010EAE000043
:00000001FF
